:100000000C94E1000C94FC000C94FC000C94FC009B
:100010000C94FC000C94FC000C94B1160C94FC00A5
:100020000C94FC000C94FC000C947E160C943F166F
:100030000C9443110C94FC000C94FC000C94FC00F8
:100040000C94FC000C941D040C94FC000C94041003
:100050000C9457100C94FC000C94FC000C94FC00C5
:100060000C94FC000C94FC000C94FC000C94FC0020
:100070004570692D4F5344205665722E302E382E10
:10008000322E310000416B7475656C6C65732053C2
:10009000657474696E67000053657474696E6720D7
:1000A000200000486F6568656E73656E736F72201F
:1000B00000004853206D697420536368616C746557
:1000C0007220000048656164696E6720486F6C6447
:1000D0002000004B6F6D706173732000004B6F6DDB
:1000E0007061737320666978200000475053204187
:1000F0006B74697620000041636873656E6B6F7086
:1001000070656C756E67200000447265687261747A
:100110006520626567722E2000004665686C657216
:100120002046433C2D3E4F5344200000556E7465DD
:10013000727370616E6E756E672000004B65696E3C
:10014000652053657474696E672D416E7A656967C1
:1001500065000050432F4254206973742065696E16
:100160006765736368616C7465740000DC62657256
:100170006E65686D65204C65747A7465732053658F
:100180007474696E6700004F4E00002D2D2D000025
:100190004550492D4D656E750050616C0050432FE0
:1001A0004254004B656E6E756E670052432D42657A
:1001B0007472696562000045786974004F4E002DC5
:1001C0002D0011241FBECFEFD4E0DEBFCDBF11E064
:1001D000A0E0B1E0E6E1F0E302C005900D92AC349E
:1001E000B107D9F713E0ACE4B1E001C01D92A0392A
:1001F000B107E1F70C9409010C94000080E981BB80
:100200008FE084BBAC9AAD9A8EE28ABBD99ADD9A14
:1002100008951F931092930110928F0110929401F0
:10022000A0E0B0E00E94F717802D9927809353013A
:10023000A1E0B0E00E94F717802D9927809300017C
:10024000A2E0B0E00E94F717802D99278093540117
:10025000A7E1B0E00E94F717802D992780936B01EA
:10026000A8E1B0E00E94F717802D992780937E01C6
:100270000E94E4150E94FE000E940D04809153012B
:10028000813019F40E94EF0F02C00E94DF0F7894B2
:10029000A89A0E94A3030E947E040E9411090E9452
:1002A0008D090E94190980914E018130B1F410929C
:1002B0004E0180919301882351F48091530188234A
:1002C00031F480916001813011F40E94F9100E9494
:1002D00036110E943B110E94E013809152019091CF
:1002E0009301813041F4992331F40E94710E0E94F0
:1002F0006B130E94C712809151018130C9F5809122
:1003000093018823A9F5AA9A0E94EF0E80916B01B0
:100310008823B9F40E94E3070E94D30680917E01EE
:1003200080FF04C00E94B6110E94ED090E943808A7
:100330000E943D0980917E0183FF19C00E94D40B69
:1003400016C080910201823054F00E9438080E9449
:100350003D090E94B6110E94ED090E94D40B8091C4
:100360000201833024F00E94E3070E94D306AA987A
:1003700080914C018130C1F5809193018823A1F5D2
:1003800010924C0180916B01882321F08091020131
:10039000833014F00E9419098091680190916901DD
:1003A0000196909369018093680180916801909112
:1003B0006901CC9769F4809166019091670101967B
:1003C0009093670180936601109269011092680111
:1003D0000E94360C0E947B0980915901813021F4E2
:1003E0000E94EA0C0E94640B10914D01113009F03B
:1003F0005ACF80919301882309F055CF10924D0177
:1004000080918401813019F0823059F406C00E9435
:10041000E80982E08093840104C00E94CB09109314
:10042000840180916B01813009F03DCF809193016F
:10043000882309F038CF80916A01813009F033CFE9
:1004400010926A0180910201813071F082301CF4B7
:10045000882339F028CF823081F0833009F023CF10
:1004600017C00E94E8091FCF0E94CB0964E084E016
:100470000E944F020E947F0416CF0E94CB0964E0C5
:1004800084E00E944F020E9411090E948D090BCF47
:100490000E94CB0964E084E00E944F02FECE482F08
:1004A000D99827E030E0DB98000000000000000051
:1004B00081E090E0022E02C0880F991F0A94E2F7B3
:1004C000842311F0DA9A01C0DA98000000000000DD
:1004D0000000DB9A000000000000000021503040C6
:1004E0008FEF2F3F3807F9F627E030E0DB98000068
:1004F00000000000000081E090E0022E02C0880FA2
:10050000991F0A94E2F7862311F0DA9A01C0DA986B
:100510000000000000000000DB9A00000000000066
:100520000000215030408FEF2F3F3807F9F6DB985D
:10053000DA98D99A089564E084E00E944F026CE44E
:1005400080E00E944F0210924E0180914E0188235C
:10055000E1F36AE08CE60E944F0260E085E00E94D1
:100560004F0208951F93CF93DF9380914C0188230E
:10057000E1F310924C010E94AB1010E00DC080918D
:100580005101813011F40E94EF0E80914C018130B5
:1005900019F410924C0111E090917F0180E0112339
:1005A00009F481E0992311F4882349F7C8E1D0E0E8
:1005B000882309F4B1C08091740380937E018091F7
:1005C0007E01DE01082E0E94FF1745E850E062E040
:1005D00082E00E94780B48E950E064E082E00E94EB
:1005E000780B43EA50E066E082E00E94780B42EB31
:1005F00050E067E082E00E94780B44EC50E068E055
:1006000082E00E94780B43ED50E069E082E00E94B6
:10061000780B4DED50E06AE082E00E94780B4BEEE3
:1006200050E06BE082E00E94780B47EF50E06CE016
:1006300082E00E94780B4CE251E06DE082E00E9483
:10064000780B40917C0150917D0164E084E10E942F
:10065000390B80917E0180FF03C047E851E002C062
:100660004BE851E066E084E10E94780B80917E01C6
:1006700081FF03C047E851E002C04BE851E067E06A
:1006800084E10E94780B80917E0182FF03C047E8DD
:1006900051E002C04BE851E068E084E10E94780B31
:1006A00080917E0183FF03C047E851E002C04BE820
:1006B00051E069E084E10E94780B80917E0184FF23
:1006C00003C047E851E002C04BE851E06AE084E132
:1006D0000E94780B80917E0185FF03C047E851E0BE
:1006E00002C04BE851E06BE084E10E94780B8091FE
:1006F0007E0186FF03C047E851E002C04BE851E0AD
:100700006CE084E10E94780B4091840355276DE0F2
:1007100084E10E94390B13C045E850E062E082E0BA
:100720000E94780B4AE151E065E082E00E94780B7C
:10073000DE010E94F717802D992780937E01DF91BB
:10074000CF911F9108950E949B0210924C018091BD
:100750004C018823E1F340E750E062E087E00E942B
:10076000780B0E947F0410924C0180914C018823E9
:10077000E1F310924C0180914C018823E1F3109237
:100780004C0164E084E00E944F026CE480E00E942F
:100790004F0280915301882319F40E94B2021AC0BB
:1007A0004CE351E062E082E00E94780B43E551E0C7
:1007B00064E082E00E94780B4CE651E066E082E063
:1007C0000E94780BA8E1B0E00E94F717802D9927CE
:1007D00080937E0180914C018823E1F310924C01BB
:1007E00080914C018823E1F310924C0180914C01DF
:1007F0008823E1F310924C0180914C018823E1F3AE
:1008000010924C0180914C018823E1F310924C012D
:1008100064E084E00E944F02089582E083BF92E486
:100820009EBD8EE189BF83E087BD86E982BD90933E
:100830008A0080E280937D0008951F920F920FB688
:100840000F9211248F939F93809150018F5F80931B
:10085000500180915001883439F591E090934F0117
:1008600010925001809188038F5F8093880380915C
:100870008803843631F41092880390934C0190934E
:100880004D0180918803823311F490934D01809142
:1008900087038F5F80938703809187038A3021F4D9
:1008A0001092870390934E019F918F910F900FBEEE
:1008B0000F901F901895282F80538A3010F090E0E9
:1008C00005C0203311F49AE001C0982F822F815483
:1008D0008A3110F4922F9653822F81568A3110F468
:1008E000922F9C532D3211F499E403C02E3209F457
:1008F00091E4892F992787FD90950895089560E0E8
:1009000085E00E944F0263E886E00E944F0260E9A2
:1009100087E00E944F0260E085E00E944F0264E899
:1009200086E00E944F0261E987E00E944F0260E08A
:1009300085E00E944F0265E886E00E944F0262E96E
:1009400087E00E944F0260E085E00E944F0266E867
:1009500086E00E944F0263E987E00E944F0260E058
:1009600085E00E944F0267E886E00E944F0264E93A
:1009700087E00E944F0260E085E00E944F0268E835
:1009800086E00E944F0265E987E00E944F0260E026
:1009900085E00E944F0269E886E00E944F0266E906
:1009A00087E00E944F0260E085E00E944F026AE803
:1009B00086E00E944F0267E987E00E944F0260E0F4
:1009C00085E00E944F0261EA86E00E944F0268E9DA
:1009D00087E00E944F0260E085E00E944F0262EAD9
:1009E00086E00E944F0269E987E00E944F0260E0C2
:1009F00085E00E944F0263EA86E00E944F026AE9A6
:100A000087E00E944F0260E085E00E944F0264EAA6
:100A100086E00E944F026BE987E00E944F0260E08F
:100A200085E00E944F0265EA86E00E944F026CE971
:100A300087E00E944F0260E085E00E944F0266EA74
:100A400086E00E944F026DE987E00E944F0260E05D
:100A500085E00E944F0267EA86E00E944F026EE93D
:100A600087E00E944F0260E085E00E944F0268EA42
:100A700086E00E944F026FE987E00E944F0260E02B
:100A800085E00E944F026FEB86E00E944F0260EA11
:100A900087E00E944F0260E085E00E944F0260EC18
:100AA00086E00E944F0261EA87E00E944F0260E008
:100AB00085E00E944F0261EC86E00E944F0262EAEC
:100AC00087E00E944F0260E085E00E944F0262ECE6
:100AD00086E00E944F0263EA87E00E944F0260E0D6
:100AE00085E00E944F0263EC86E00E944F0264EAB8
:100AF00087E00E944F0260E085E00E944F0264ECB4
:100B000086E00E944F0265EA87E00E944F0260E0A3
:100B100085E00E944F0265EC86E00E944F0266EA83
:100B200087E00E944F0260E085E00E944F0266EC81
:100B300086E00E944F0267EA87E00E944F0260E071
:100B400085E00E944F026DED86E00E944F0268EA48
:100B500087E00E944F0260E085E00E944F026EED48
:100B600086E00E944F0269EA87E00E944F0260E03F
:100B700085E00E944F026FED86E00E944F026AEA14
:100B800087E00E944F0260E085E00E944F0260EE25
:100B900086E00E944F026BEA87E00E944F0260E00D
:100BA00085E00E944F0261EE86E00E944F026CEAEF
:100BB00087E00E944F0260E085E00E944F0262EEF3
:100BC00086E00E944F026DEA87E00E944F0260E0DB
:100BD00085E00E944F0263EE86E00E944F026EEABB
:100BE00087E00E944F0260E085E00E944F0264EEC1
:100BF00086E00E944F026FEA87E00E944F0260E0A9
:100C000085E00E944F026BEF86E00E944F0260EB8E
:100C100087E00E944F0260E085E00E944F026CEF87
:100C200086E00E944F0261EB87E00E944F0260E085
:100C300085E00E944F026DEF86E00E944F0262EB5A
:100C400087E00E944F0260E085E00E944F026EEF55
:100C500086E00E944F0263EB87E00E944F0260E053
:100C600085E00E944F026FEF86E00E944F0264EB26
:100C700087E00E944F0261E085E00E944F0260E041
:100C800086E00E944F0265EB87E00E944F0261E020
:100C900085E00E944F0261E086E00E944F0266EB11
:100CA00087E00E944F020895FF920F931F93CF9306
:100CB000DF938C01F62EEC0117C06D2F772785E0AE
:100CC0000E944F026C2F86E00E944F028F2D9927C1
:100CD000FC01EE0FFF1FE80FF91FE15FFE4F60817F
:100CE00087E00E944F022196C8010596C817D907D0
:100CF00020F3E8012A9617C06D2F772785E00E9420
:100D00004F026C2F86E00E944F028F2D9927FC0125
:100D1000EE0FFF1FE80FF91FE15FFE4F608187E0D4
:100D20000E944F022196C8010F96C817D90720F3D9
:100D3000DF91CF911F910F91FF9008950F931F9313
:100D4000CF93DF938C01EC010EC06D2F772785E0E8
:100D50000E944F026C2F86E00E944F0260E087E005
:100D60000E944F022196C8010596C817D90768F35B
:100D7000E8012A960EC06D2F772785E00E944F026A
:100D80006C2F86E00E944F0260E087E00E944F02D5
:100D90002196C8010F96C817D90768F3DF91CF9144
:100DA0001F910F9108951F93CF93DF938091280394
:100DB0009091290366E170E00E94C2179B012E5FAB
:100DC0003F4F37FD1BC0C9016AE070E00E94C217A7
:100DD000182F1695C9016AE070E00E94C21787E0DB
:100DE00090E0861B91092EE130E0829FE001839F15
:100DF000D00D929FD00D1124279616C030952195C5
:100E00003F4FC9016AE070E00E94C217182F169583
:100E10001C5FC9016AE070E00E94C2178EE1689F02
:100E2000E0011124C950DF4F80910B0190910C011A
:100E3000C817D90739F080910B0190910C010E94DD
:100E40009E0604C080918201811721F0612FCE019E
:100E50000E94540610938201D0930C01C0930B01A1
:100E6000DF91CF911F910895AF92BF92DF92EF92E1
:100E7000FF920F931F93CF93DF93CDB7DEB72197E8
:100E80000FB6F894DEBF0FBECDBF8C01D62E5C012D
:100E900019826B2D772785E00E944F026A2D86E02C
:100EA0000E944F02ED2CFF24F701E35DFE4F6081AD
:100EB00087E00E944F028EE190E0A80EB91E998152
:100EC000925E99839C3329F7F4EBAF2EB12CA00EE0
:100ED000B11E6B2D772785E00E944F026A2D86E0B8
:100EE0000E944F02F701E35DFE4F608187E00E94A0
:100EF0004F02EEE1F0E0AE0EBF1EC801825F9E4FD2
:100F0000A816B90631F721960FB6F894DEBF0FBECA
:100F1000CDBFDF91CF911F910F91FF90EF90DF90A8
:100F2000BF90AF900895EF92FF920F931F93CF93CE
:100F3000DF93CDB7DEB721970FB6F894DEBF0FBEB3
:100F4000CDBF8C017C0119826F2D772785E00E942F
:100F50004F026E2D86E00E944F0260E087E00E9403
:100F60004F028EE190E0E80EF91E9981925E99831E
:100F70009C3351F784EBE82EF12CE00EF11E6F2D1F
:100F8000772785E00E944F026E2D86E00E944F0277
:100F900060E087E00E944F02EEE1F0E0EE0EFF1EFF
:100FA000C801825F9E4FE816F90649F721960FB6F1
:100FB000F894DEBF0FBECDBFDF91CF911F910F918F
:100FC000FF90EF9008951F93CF93DF9380912A03B2
:100FD00090912B0366E170E00E94C2179B012A5F8B
:100FE0003F4F37FD12C0C9016AE070E00E94C2178E
:100FF000182F16951C5FC9016AE070E00E94C217A5
:10100000C6E8D0E0C61BD10913C0309521953F4FEB
:10101000C9016AE070E00E94C217182F1695C90135
:101020006AE070E00E94C217C62FDD27C957DF4F64
:1010300080910D0190910E01C817D90739F0809168
:101040000D0190910E010E94930704C080918301CD
:10105000811721F0612FCE010E9434071093830184
:10106000D0930E01C0930D01DF91CF911F91089590
:10107000FF920F931F93CF93DF9380913A03909148
:101080003B038E55904063E070E00E94C217EB0175
:101090006A3071051CF0C9E0D0E004C077FF02C0DF
:1010A000C0E0D0E08091640190916501C817D90734
:1010B00009F47DC0C230D10514F468E101C068E0D4
:1010C00084E00E944F02D0936501C0936401C53053
:1010D000D105B9F1C630D1057CF4C230D10521F17A
:1010E000C330D1051CF42197A9F419C0C330D10530
:1010F00001F1249779F421C0C730D10549F1C730F7
:10110000D1051CF1C830D10531F1299719F4BBE89C
:10111000FB2E23C0A8E8FA2E04E810E820C0F8E867
:10112000FF2E04E811E81BC0E8E8FE2E04E812E8F0
:1011300016C078E8F72E04E811C068E8F62E05E836
:101140000DC058E8F52E06E809C048E8F42E05C0A1
:1011500039E8F32E02C02AE8F22E07E813E860E02F
:1011600085E00E944F026FE186E00E944F02612FEE
:1011700087E00E944F0260E085E00E944F026DE32D
:1011800086E00E944F02602F87E00E944F0260E0DD
:1011900085E00E944F026BE586E00E944F026F2DB2
:1011A00087E00E944F0260E084E00E944F02DF91DE
:1011B000CF911F910F91FF900895EF92FF920F939F
:1011C0001F93CF93DF937A019EE1699FB0011124B1
:1011D000680F711D8B01020F111D10928903EB0125
:1011E00016C06D2F772785E00E944F026C2F86E096
:1011F0000E944F0280918903F701E80FF11D608181
:101200008F5F8093890387E00E944F022196C01769
:10121000D10738F3DF91CF911F910F91FF90EF909D
:10122000089525E046E051E06EE081E00E94DD088F
:101230000895CF93DF93CDB7DEB725970FB6F89417
:10124000DEBF0FBECDBFDE011196EAE3F1E085E01F
:1012500001900D928150E1F725E0AE014F5F5F4FA5
:1012600067E08CE00E94DD0825960FB6F894DEBF9B
:101270000FBECDBFDF91CF910895CF93DF93CDB750
:10128000DEB724970FB6F894DEBF0FBECDBF19822C
:101290001A8285E48B831C8230913A03832F6AE0A3
:1012A0000E94A217282F0E94A217482F822F0E9467
:1012B000A217292F832F0E94A217992319F48AE0DD
:1012C0008C8301C09C83222319F48AE08A8301C0A5
:1012D0002A83498324E0AE014F5F5F4F61E083E0E2
:1012E0000E94DD0824960FB6F894DEBF0FBECDBF76
:1012F000DF91CF91089580915401813069F420915C
:10130000A101922F27FD9F5F959542EA51E061E090
:101310008EE0891B0E94DD08089560E085E00E9450
:101320004F026FE186E00E944F0260E887E00E9472
:101330004F0260E085E00E944F026DE386E00E946C
:101340004F0264E887E00E944F0260E085E00E945F
:101350004F026BE586E00E944F0268E887E00E943A
:101360004F02089560E085E00E944F026FEC86E036
:101370000E944F026CE887E00E944F0261E085E026
:101380000E944F026BE086E00E944F026DE887E00A
:101390000E944F0208956CE480E00E944F0208957D
:1013A00080913C0390913D03843B910544F48091EE
:1013B0008401882361F481E0809384010895809101
:1013C0008401181614F40E94CB0910928401089528
:1013D00062E480E00E944F020895EF92FF920F9323
:1013E0001F93CF93DF93CDB7DEB72F970FB6F89447
:1013F000DEBF0FBECDBF85E0FE01369611928A9505
:10140000E9F780913203909133036EE170E00E941E
:10141000C217CB018E01055F1F4F019797FF02C0D6
:1014200080E090E04AE050E0B8010E947117F801B6
:1014300001900020E9F73197EE2EE01A109289030F
:10144000FF240AC00E0F1F1FEC0FFD1F83850E9493
:101450005B04F8018083F394EF2DFF278E2D9927ED
:1014600087FD90958E010F5F1F4FE817F90754F322
:10147000F092890325E0AE014A5F5F4F69E085E1A4
:101480000E94DD082E2DA80169E089E18E190E94D5
:10149000DD082F960FB6F894DEBF0FBECDBFDF91EB
:1014A000CF911F910F91FF90EF900895EF92FF92CF
:1014B0000F931F93CF93DF93CDB7DEB72E970FB661
:1014C000F894DEBF0FBECDBF19821A821B821C8228
:1014D00080917401909175018E01065F1F4F4AE063
:1014E00050E0B8010E947117F80101900020E9F75F
:1014F0003197EE2EE01A10928903FF240AC00E0FD6
:101500001F1FEC0FFD1F82850E945B04F801808382
:10151000F394EF2DFF278E2D992787FD90958E014F
:101520000B5F1F4FE817F90754F3F092890324E08B
:10153000AE014F5F5F4F66E085E10E94DD082E2D12
:10154000A80166E089E18E190E94DD08809174018E
:10155000909175011816190664F460E085E00E9408
:101560004F0262EC86E00E944F026CE887E00E9426
:101570004F02809174019091750197FF0CC060E05B
:1015800085E00E944F0262EC86E00E944F026DE807
:1015900087E00E944F028091740190917501892B20
:1015A00061F460E085E00E944F0262EC86E00E94F8
:1015B0004F0260E087E00E944F022E960FB6F8942B
:1015C000DEBF0FBECDBFDF91CF911F910F91FF9076
:1015D000EF9008959F92AF92BF92CF92DF92EF92D9
:1015E000FF920F931F93CF93DF93CDB7DEB76E9724
:1015F0000FB6F894DEBF0FBECDBF982EA62E7A018F
:10160000FA0101900020E9F73197BE2EB41ACC24DC
:10161000DD240BC0FF278A010E0F1F1FEE0DFF1DDB
:1016200080810E945B04F8018083EC2D0894C11C2A
:10163000D11C8B2D99270196AE014F5F5F4FC816C5
:10164000D90641F72B2D6A2D892D0E94DD086E9653
:101650000FB6F894DEBF0FBECDBFDF91CF911F91C3
:101660000F91FF90EF90DF90CF90BF90AF909F9041
:101670000895EF92FF920F931F93CF93DF93CDB70F
:10168000DEB764970FB6F894DEBF0FBECDBFE82E6D
:10169000F62ECA014AE050E08E010F5F1F4FB801DD
:1016A0000E947117A8016F2D8E2D0E94EA0A649680
:1016B0000FB6F894DEBF0FBECDBFDF91CF911F9163
:1016C0000F91FF90EF90089560915C0170915D0122
:1016D00080915E0190915F0128E631E040E050E0AA
:1016E0000E94D517A90163E083E00E94390B089599
:1016F000BF92CF92DF92EF92FF920F931F93CF93FF
:10170000DF93CDB7DEB764970FB6F894DEBF0FBE98
:10171000CDBFB82EC62E9A01DE01119605C0EA0F84
:10172000FB1F90832F5F3F4F822F841BF901949101
:10173000E82FFF27992399F7EA0FFB1F1082FD017D
:1017400001900020E9F73197DE2EDA1AEE24FF240B
:1017500009C08D01020F111DF80180810E945B04F8
:10176000F80180832E2D0894E11CF11C8D2D992702
:101770000196DE011196E816F90659F72D2DAD01F7
:101780006C2D8B2D0E94DD0864960FB6F894DEBF99
:101790000FBECDBFDF91CF911F910F91FF90EF90C2
:1017A000DF90CF90BF900895EF92FF920F931F9319
:1017B000CF93DF93CDB7DEB72B970FB6F894DEBF8C
:1017C0000FBECDBFDE011196E7E3F1E083E00190AB
:1017D0000D928150E1F78E01085F1F4F4AE050E003
:1017E000B80180913803909139030E947117F80174
:1017F00001900020E9F73197EE2EE01A109289034C
:10180000FF240AC00E0F1F1FEC0FFD1F80850E94D2
:101810005B04F8018083F394EF2DFF278E2D992729
:1018200087FD90958E010C5F1F4FE817F90754F361
:10183000F092890323E0AE014F5F5F4F6EE08DE0D1
:101840000E94DD082E2DA8016EE080E18E190E9415
:10185000DD082B960FB6F894DEBF0FBECDBFDF912B
:10186000CF911F910F91FF90EF900895EF92FF920B
:101870000F931F93CF93DF93CDB7DEB728970FB6A3
:10188000F894DEBF0FBECDBF19828AE08A838091B3
:101890006601909167018E010A5F1F4F4AE050E098
:1018A000B8010E947117F80101900020E9F7319703
:1018B000EE2EE01A10928903FF240DC08E010D5FF9
:1018C0001F4F0E0F1F1FEC0FFD1F86810E945B0430
:1018D000F8018083F394EF2DFF278E2D992787FD44
:1018E0009095E817F90754F3F09289038091660107
:1018F000909167018E010D5F1F4F0A976CF421E0F4
:10190000AE014F5F5F4F6EE081E00E94DD0821E095
:10191000A8016EE082E004C022E0A8016EE081E050
:101920000E94DD0880916801909169018E010A5F33
:101930001F4F4AE050E0B8010E947117F801019072
:101940000020E9F73197EE2EE01A10928903FF2468
:101950000DC08E010D5F1F4F0E0F1F1FEC0FFD1FDF
:1019600086810E945B04F8018083F394EF2DFF27AA
:101970008E2D992787FD9095E817F90754F3F0927B
:10198000890380916801909169018E010D5F1F4F5D
:101990000A976CF421E0AE014E5F5F4F6EE084E089
:1019A0000E94DD0821E0A8016EE085E004C022E08D
:1019B000A8016EE084E00E94DD0828960FB6F89436
:1019C000DEBF0FBECDBFDF91CF911F910F91FF9072
:1019D000EF900895CF92DF92EF92FF920F931F93B3
:1019E000CF93DF93CDB7DEB72B970FB6F894DEBF5A
:1019F0000FBECDBF80915A0190915B0180915A0139
:101A000090915B018D5A964230F08CEA96E2909369
:101A10005B0180935A0180915A0190915B0164E6C9
:101A200070E00E94AE17709356016093550180914B
:101A30005A0190915B0164E670E00E94AE179093AA
:101A400058018093570180915701909158016AE0A5
:101A500070E00E94AE177093580160935701809117
:101A600055019091560125E429831A821B828E012B
:101A7000085F1F4F4AE050E0B8010E947117F8015B
:101A800001900020E9F73197CE2EC01A10928903F9
:101A9000DD240BC0020F131FE20EF31EF70180813D
:101AA0000E945B04F8018083D3942D2D33278C2D65
:101AB000992787FD909548E0E42EF12CEC0EFD1E51
:101AC0008E010C5F1F4F2817390724F3D09289032A
:101AD00022E0AE014E5F5F4F62E083E00E94DD08CE
:101AE0002C2DA80162E085E08C190E94DD08809110
:101AF0005701909158014AE050E0B7010E947117D8
:101B0000F70101900020E9F73197EE19EE2E1092BF
:101B10008903FF240AC00E0F1F1FEC0FFD1F8085D5
:101B20000E945B04F8018083F394EF2DFF278E2D34
:101B3000992787FD90958E010C5F1F4FE817F907D5
:101B400054F3F092890321E0AE014F5F5F4F62E0F2
:101B500085E00E94DD0821E0AE014E5F5F4F62E04C
:101B600086E00E94DD0821E0A80162E086E00E9494
:101B7000DD082B960FB6F894DEBF0FBECDBFDF9108
:101B8000CF911F910F91FF90EF90DF90CF9008952C
:101B90000F931F93CF93DF93CDB7DEB72A970FB67E
:101BA000F894DEBF0FBECDBF4AE050E08E010F5F5C
:101BB0001F4FB8010E947117F80101900020E9F74A
:101BC0003197E01B1092890320E0FF27E7FDF09595
:101BD00001C02F5F822F99278E179F07D4F3209380
:101BE00089032A960FB6F894DEBF0FBECDBFDF91F2
:101BF000CF911F910F9108950F931F93CF93DF9370
:101C000060E070E0C3E0D0E0A3E9B2E03C91FD0108
:101C1000218112810381CE010496EC011496835D2B
:101C2000924009F459C0422F55274D535040E0913E
:101C30004301F0914401E60FF71F832F9927CD97B9
:101C4000880F991F880F991F9A01689413F835958A
:101C500027951694E1F7822B932B808368317105C9
:101C6000D9F1212F33272D533040FB01319680913C
:101C7000430190914401E80FF91F4F70507084E0C8
:101C8000440F551F8A95E1F7C9019595879595955C
:101C90008795482B592B408381E067317807E1F025
:101CA000FB0132968091430190914401E80FF91FA6
:101CB0002370307086E0220F331F8A95E1F7802F62
:101CC0009927CD97282B392B2083E2E066317E07B8
:101CD00019F06D5F7F4F9ACFDF91CF911F910F91D8
:101CE0000895EF92FF920F931F93CF93DF9380910C
:101CF000B801843409F06AC033E0E32EF12C60E0CF
:101D000070E0A9EBB1E08C91FD012181128103818A
:101D1000E70124967E0114966134710509F456C0DA
:101D2000422F55274D535040E0914101F09142011F
:101D3000E60FF71F9927CD97880F991F880F991FD6
:101D40009A01689413F8359527951694E1F7822B3C
:101D5000932B808360347105C9F1212F33272D53D4
:101D60003040FB0131968091410190914201E80F92
:101D7000F91F4F70507084E0440F551F8A95E1F7AA
:101D8000C9019595879595958795482B592B408343
:101D9000CB35D105D9F0FB0132968091410190916C
:101DA0004201E80FF91F2370307046E0220F331F05
:101DB0004A95E1F7802F9927CD97282B392B20833F
:101DC0006E33710519F06D5F7F4F9DCF10925201F8
:101DD000DF91CF911F910F91FF90EF900895EF92B7
:101DE000FF920F931F93CF93DF93809192028434DD
:101DF00009F091C033E0E32EF12C60E070E0A3E93C
:101E0000B2E08C91FD01218112810381E7012496CA
:101E10007E0114966134710509F456C0422F55278E
:101E20004D535040E0913F01F0914001E60FF71F04
:101E30009927CD97880F991F880F991F9A01689449
:101E400013F8359527951694E1F7822B932B808311
:101E500060347105C9F1212F33272D533040FB0128
:101E6000319680913F0190914001E80FF91F4F702A
:101E7000507084E0440F551F8A95E1F7C90195958C
:101E8000879595958795482B592B4083CB35D10560
:101E9000D9F0FB01329680913F0190914001E80F0B
:101EA000F91F2370307046E0220F331F4A95E1F787
:101EB000802F9927CD97282B392B20836E337105DE
:101EC00019F06D5F7F4F9DCF80913C0390913D0352
:101ED000843B91058CF4809160018130E1F4109293
:101EE0006001F8940E94EF0F789480913C039091E8
:101EF0003D03843B91057CF080916001882359F477
:101F000081E080936001F89480915301882311F45B
:101F10000E94DF0F7894809192028C3459F481E012
:101F200090E090937D0180937C0181E080937F011C
:101F30000E94FC0D809192028D3459F482E090E071
:101F400090937D0180937C0181E080937F010E94CA
:101F5000FC0D809192028E3459F483E090E09093CE
:101F60007D0180937C0181E080937F010E94FC0DC4
:101F7000809192028F3459F484E090E090937D0137
:101F800080937C0181E080937F010E94FC0D809111
:101F90009202803559F485E090E090937D01809322
:101FA0007C0181E080937F010E94FC0D1092510121
:101FB000DF91CF911F910F91FF90EF90089582E2F2
:101FC00089B910BC80B91CBE909A28E92AB996E854
:101FD00090BD82EC8BB921B99CBF82B9089582E291
:101FE00089B910BC80B91CBE909A88E98AB926E8E4
:101FF00020BD92EC9BB980E981B92CBF92B90895BC
:10200000159BFECF83B908951F920F920FB60F92C2
:1020100011248F939F93EF93FF939CB190938A0326
:102020009D3081F480918601813061F4AB981092EB
:10203000860180935201E0916B03FF27EA54FE4F23
:1020400090832CC080918601882319F0813031F56E
:1020500013C0933239F480915201882319F481E03E
:102060008093860110926B0380916B03E82FFF270A
:10207000EA54FE4F90830CC0E0916B03FF27EA54B3
:10208000FE4F908380916B03853930F480916B0310
:102090008F5F80936B0302C010928601FF91EF91D6
:1020A0009F918F910F900FBE0F901F9018951F92C8
:1020B0000F920FB60F9211248F939F93EF93FF937C
:1020C00093B190938B039D3081F480918501813091
:1020D00061F4AB981092850180935101E0916803FF
:1020E000FF27E057FD4F90832DC080918501882305
:1020F00019F0813039F514C0933241F480915101C7
:10210000882321F481E080938501AB9A10926803C3
:1021100080916803E82FFF27E057FD4F90830CC0A4
:10212000E0916803FF27E057FD4F9083809168039B
:10213000853930F4809168038F5F8093680302C013
:1021400010928501FF91EF919F918F910F900FBE9B
:102150000F901F901895CF93DF93CDB7DEB72C97D4
:102160000FB6F894DEBF0FBECDBF83E289831A821B
:1021700081E78B838CE78C838DE68D838DE38E8363
:102180008F8320E030E0FE013196AE01485F5F4F63
:102190008191280F311DE417F507D1F7C90160E0DF
:1021A00070E10E94C2179C0160E470E00E94C217B7
:1021B000635C6887C90160E470E00E94C217835CB9
:1021C00089878DE08A87FE0131969E01255F3F4F0A
:1021D0008081159BFECF83B93196E217F307C1F7D3
:1021E0002C960FB6F894DEBF0FBECDBFDF91CF9116
:1021F0000895CF93DF93CDB7DEB72A970FB6F89443
:10220000DEBF0FBECDBF83E289831A8283E68B8354
:102210001C821D8286E890E060E070E10E94C21797
:102220009C0160E470E00E94C217635C6E83C90188
:1022300060E470E00E94C217835C8F838DE0888722
:10224000FE0131969E01275F3F4F8081159BFECF97
:1022500083B93196E217F307C1F72A960FB6F894BF
:10226000DEBF0FBECDBFDF91CF91089585B392E061
:10227000892785BB089590916301913019F485B346
:10228000892785BB08951F920F920FB60F921124D4
:102290002F933F935F936F937F938F939F93AF930E
:1022A000BF938091870190918801892B81F484B537
:1022B00095B590938E0180938D018EB58F7B8EBDE9
:1022C00081E090E0909388018093870141C084B5BC
:1022D00095B590938C0180938B012EB520642EBD13
:1022E00020918D0130918E01821B930B10928801F9
:1022F00010928701865698406CE271E00E94AE17FA
:1023000070938A016093890177FF05C010928A015A
:102310001092890109C06730710534F086E090E0C1
:1023200090938A01809389012091890130918A01DB
:1023300080910201992787FD90952817390741F070
:10234000263031052CF42093020181E080936A014C
:10235000BF91AF919F918F917F916F915F913F91CD
:102360002F910F900FBE0F901F9018958091320300
:102370009091330390936D0180936C0180916C0177
:1023800090916D0120916E0130916F01821B930B32
:10239000909371018093700180916C0190916D0117
:1023A00090936F0180936E01409178015091790173
:1023B0002091700130917101CA01E3E0880F991FEB
:1023C000EA95E1F7841B950B73E0220F331F7A9592
:1023D000E1F7820F931F68E070E00E94C2177093CC
:1023E00079016093780120917A0130917B014091CD
:1023F000780150917901C90163E0880F991F6A95AE
:10240000E1F7821B930B840F951F68E070E00E9438
:10241000C21770937B0160937A0180917A01909149
:102420007B0190937501809374010E94560A089570
:10243000BF92CF92DF92EF92FF920F931F93CF93B1
:10244000DF93CDB7DEB760970FB6F894DEBF0FBE4F
:10245000CDBF19821A821B821C82809184029091C6
:10246000850290938F0380938E03809186029091D2
:10247000870290938D0380938C0380918E039091BB
:102480008F038E01055F1F4F4AE050E0B8010E94A4
:102490007117F80101900020E9F73197BE2EB01AAC
:1024A000CC24DD240DC0EC0CFD1CF70180810E94C2
:1024B0005B040C0D1D1DF80180830894C11CD11C08
:1024C0008B2D992787FD90952BE0E22EF12CEC0EB9
:1024D000FD1E8E010B5F1F4FC816D90624F324E0A2
:1024E000AE014F5F5F4F61E08CE00E94DD082B2D55
:1024F000A80161E080E18B190E94DD0880918C03C6
:1025000090918D034AE050E0B7010E947117F701E6
:1025100001900020E9F73197DE2EDE18EE24FF242B
:102520000DC0FE01EE0DFF1D83850E945B040E0DA4
:102530001F1DF80180830894E11CF11C8D2D992743
:1025400087FD90958E010B5F1F4FE816F9064CF33F
:1025500024E0AE014F5F5F4F62E08CE00E94DD0837
:102560002D2DA80162E080E18D190E94DD086096A2
:102570000FB6F894DEBF0FBECDBFDF91CF911F9194
:102580000F91FF90EF90DF90CF90BF9008958F92C2
:102590009F92BF92CF92DF92EF92FF920F931F9381
:1025A000CF93DF93CDB7DEB760970FB6F894DEBF59
:1025B0000FBECDBF19821A821B821C8280904C03F1
:1025C00090904D038E01055F1F4F4AE050E0B80127
:1025D00080914A0390914B030E947117F80101907A
:1025E0000020E9F73197BE2EB01ACC24DD240DC0AF
:1025F000EC0CFD1CF70180810E945B040C0D1D1D7D
:10260000F80180830894C11CD11C8B2D992787FD6C
:1026100090953BE0E32EF12CEC0EFD1E8E010B5F3E
:102620001F4FC816D90624F324E0AE014F5F5F4F59
:1026300064E08CE00E94DD082B2DA80164E080E1BD
:102640008B190E94DD084AE050E0B701C4010E94E6
:102650007117F70101900020E9F73197DE2EDE189F
:10266000EE24FF240DC0FE01EE0DFF1D83850E94A8
:102670005B040E0D1F1DF80180830894E11CF11C02
:102680008D2D992787FD90958E010B5F1F4FE816C2
:10269000F9064CF324E0AE014F5F5F4F65E08CE03C
:1026A0000E94DD082D2DA80165E080E18D190E94B2
:1026B000DD0860960FB6F894DEBF0FBECDBFDF9188
:1026C000CF911F910F91FF90EF90DF90CF90BF902F
:1026D0009F908F900895DF92EF92FF920F931F9338
:1026E000CF93DF93CDB7DEB72B970FB6F894DEBF4D
:1026F0000FBECDBFDE011196E9E4F1E083E0019069
:102700000D928150E1F78E01085F1F4F4AE050E0C3
:10271000B80180918C0290918D020E947117F8018E
:1027200001900020E9F73197DE2ED01AEE24FF2425
:102730000DC0FE01EE0DFF1D80850E945B040E0D95
:102740001F1DF80180830894E11CF11C8D2D992731
:1027500087FD90958E010C5F1F4FE816F9064CF32C
:1027600023E0AE014F5F5F4F61E088E10E94DD082A
:102770002D2DA80161E08BE18D190E94DD082B96BB
:102780000FB6F894DEBF0FBECDBFDF91CF911F9182
:102790000F91FF90EF90DF90089522E047E451E021
:1027A00061E08AE10E94DD080895F89488E190E0F4
:1027B00028E00FB6F894A89581BD0FBE21BDFFCFCC
:1027C0001F939D9902C180918F018F5F80938F012C
:1027D00091E09093910180918F01853009F0F9C0CB
:1027E00080919301882309F071C090939301109216
:1027F000940164E084E00E944F022091A10142EA2A
:1028000051E061E083E00E94DD0840E951E063E0CF
:1028100083E00E94780B68E084E00E944F0249E95F
:1028200051E065E083E00E94780B809100018130E7
:1028300019F44CEB51E002C04FEB51E065E084E14C
:102840000E94780B60E084E00E944F024DE951E065
:1028500066E083E00E94780B80915301813019F487
:102860004CEB51E002C04FEB51E066E084E10E9486
:10287000780B43EA51E067E083E00E94780B809197
:102880005401813019F44CEB51E002C04FEB51E0A0
:1028900067E084E10E94780B4BEA51E068E083E056
:1028A0000E94780B80916B01813019F44CEB51E060
:1028B00002C04FEB51E068E084E10E94780B47EBE7
:1028C00051E06BE083E00E94780B81C0109194018D
:1028D000113001F568E084E00E944F0280915301BD
:1028E000882329F4109353014CEB51E004C010925B
:1028F00053014FEB51E066E084E10E94780B809138
:102900005301A0E0B0E0082E0E94FF1760E084E0D1
:102910000E944F0280919401823009F568E084E0C2
:102920000E944F0280915401882331F481E080930A
:1029300054014CEB51E004C0109254014FEB51E0B4
:1029400067E084E10E94780B80915401A2E0B0E03E
:10295000082E0E94FF1760E084E00E944F028091E1
:102960009401833009F568E084E00E944F02809171
:102970006B01882331F481E080936B014CEB51E0D3
:1029800004C010926B014FEB51E068E084E10E94BB
:10299000780B80916B01A7E1B0E0082E0E94FF1731
:1029A00060E084E00E944F0280919401843089F4B9
:1029B00010929301F89488E190E028E00FB6F89423
:1029C000A89581BD0FBE21BDFFCF10928F0110923F
:1029D00091019C99E9C090919301913009F0EAC06E
:1029E00090939201809190018F5F809390018091EC
:1029F0009001853009F0DEC0109290018091940121
:102A0000823009F464C0833030F4882359F0813077
:102A100009F0D0C031C0833009F483C0843009F09C
:102A2000C9C09EC09093940149E951E065E083E0FC
:102A30000E94780B80910001813019F44CEB51E039
:102A400002C04FEB51E065E084E10E94780B68E042
:102A500084E00E944F024DE951E066E083E00E946D
:102A6000780B80915301813019F44CEB51E002C096
:102A70004FEB51E066E090C082E0809394014DE915
:102A800051E066E083E00E94780B80915301813031
:102A900019F44CEB51E002C04FEB51E066E084E1E9
:102AA0000E94780B68E084E00E944F0243EA51E004
:102AB00067E083E00E94780B80915401813019F423
:102AC0004CEB51E002C04FEB51E067E065C083E0A2
:102AD0008093940143EA51E067E00E94780B809173
:102AE0005401813019F44CEB51E002C04FEB51E03E
:102AF00067E084E10E94780B68E084E00E944F0266
:102B00004BEA51E068E083E00E94780B80916B0112
:102B1000813019F44CEB51E002C04FEB51E068E01A
:102B20003BC084E0809394014BEA51E068E083E08D
:102B30000E94780B80916B01813019F44CEB51E0CD
:102B400002C04FEB51E068E084E10E94780B68E03E
:102B500084E00E944F0247EB51E06BE083E01DC030
:102B60001092940147EB51E06BE083E00E94780BF8
:102B700068E084E00E944F0249E951E065E083E0AB
:102B80000E94780B80910001813019F44CEB51E0E8
:102B900002C04FEB51E065E084E10E94780B60E0F9
:102BA00084E00E944F0206C0109290018091910132
:102BB000809192011F910895813029F4A0E0B0E046
:102BC000062E0E94FF170895EF92FF920F931F9316
:102BD000CF93DF93CDB7DEB764970FB6F894DEBF1F
:102BE0000FBECDBF40E050E08E010F5F1F4F842F1E
:102BF0009927DC01AD5FBF4F0E94F717202D3327C7
:102C0000F801E80FF91F20832223F1F04F5F5F4F97
:102C10002F3F69F7108218C0FE01E00FF11F81817C
:102C20000E945B040E551E4FF80180830E2D112764
:102C30000894E11CF11C8091A101992787FD9095D2
:102C4000081719074CF30EC0DE011196FD01019023
:102C50000020E9F73197EA1BFB0BE093A101EE247A
:102C6000FF24E4CF64960FB6F894DEBF0FBECDBF4D
:102C7000DF91CF911F910F91FF90EF9008951F92D8
:102C80000F920FB60F9211248F939F93809198010A
:102C90008130A1F0813018F0823049F525C0809153
:102CA00096018E3129F41092960181E0809398016B
:102CB000809196018F5F8093960119C09091970142
:102CC000923061F41092970180919501813019F44E
:102CD0009093980103C083E08093980180919701BD
:102CE0008F5F8093970103C083E0809398019F9149
:102CF0008F910F900FBE0F901F9018951F920F92FB
:102D00000FB60F9211248F9380919801833011F4A4
:102D1000109298018F910F900FBE0F901F901895F1
:102D2000809128039091290365E070E00E94C2170A
:102D300066507F4F77FD0FC081E0653F78071CF03C
:102D400064EF71E003C06B3F71053CF06A5F81E0A6
:102D50008093950104C060E070E01092950162BD1F
:102D600008951F920F920FB60F921124EF92FF92C7
:102D70000F931F932F933F934F935F936F937F9383
:102D80008F939F93AF93BF93EF93FF9321E0209393
:102D9000590180919901882381F48091800090915C
:102DA00081009093A00180939F0180918A008F7B86
:102DB00080938A00209399017FC080918000909138
:102DC000810090935B0180935A0180918A00806416
:102DD00080938A00109289001092880010929901C5
:102DE00080915A0190915B0120919F013091A00147
:102DF000821B930B90935B0180935A0180915A013F
:102E000090915B019695879590935B0180935A0111
:102E100080915A0190915B018456904090935B01A0
:102E200080935A0180915A0190915B019C01442743
:102E3000552780919A0190919B01A0919C01B0919E
:102E40009D01280F391F4A1F5B1F20939A01309361
:102E50009B0140939C0150939D0180919E01843180
:102E600030F110929E01E0905C01F0905D010091C4
:102E70005E0110915F01CA01B90124E130E040E038
:102E800050E00E94D517E20EF31E041F151FE092BA
:102E90005C01F0925D0100935E0110935F0110925E
:102EA0009A0110929B0110929C0110929D018091B9
:102EB0009E018F5F80939E01FF91EF91BF91AF9133
:102EC0009F918F917F916F915F914F913F912F9142
:102ED0001F910F91FF90EF900F900FBE0F901F90DA
:102EE0001895FB019F01E8944230C4F04532B4F4D8
:102EF0004A3029F497FB1EF4909581959F4F642FDB
:102F000077270E94AE17805D8A330CF0895D81932C
:102F1000CB010097A1F716F45DE251931082C9012D
:102F20000C949217DC01FC0101900020E9F7329724
:102F3000AE17BF0730F47C916081708331976D9339
:102F4000F7CF0895991B79E004C0991F961708F0F0
:102F5000961B881F7A95C9F780950895AA1BBB1BFD
:102F600051E107C0AA1FBB1FA617B70710F0A61B89
:102F7000B70B881F991F5A95A9F780959095BC01AA
:102F8000CD01089597FB092E07260AD077FD04D0BE
:102F9000E5DF06D000201AF4709561957F4F089503
:102FA000F6F7909581959F4F0895A1E21A2EAA1BDE
:102FB000BB1BFD010DC0AA1FBB1FEE1FFF1FA217E9
:102FC000B307E407F50720F0A21BB30BE40BF50BE6
:102FD000661F771F881F991F1A9469F7609570956F
:102FE000809590959B01AC01BD01CF010895E199B9
:102FF000FECFBFBBAEBBE09A11960DB20895E1992A
:10300000FECFBFBBAEBB0DBA11960FB6F894E29AD5
:06301000E19A0FBE0895D5
:1030160001010200000A00004400002300230054BE
:1030260064665363655262005161005060005060EF
:1030360000516100526200536365546466676869B3
:103046006A6B6B6A696867000000535363535326C3
:0C305600034C026C030D0A0A1D00000070
:00000001FF
